:100000000C9466020C94AD020C94AD020C94AD02FB
:100010000C94AD020C94AD020C94AD020C94AD02A4
:100020000C94AD020C94AD020C94320C0C94040DA3
:100030000C94AD020C94AD020C94AD020C94AD0284
:100040000C94AD020C9478210C94AD020C94AD028A
:100050000C94AD020C940A1B0C94AD020C94AD02EE
:100060000C94AD020C94AD020C94AD020C94AD0254
:100070000C94AD020C94AD020C94AD020C94AD0244
:100080000C94AD020C94AD020C94AD020C94AD0234
:100090000C94AD020C94AD020C94AD020C94AD0224
:1000A0000C94AD020C94AD020C94AD02710D930D45
:1000B000860E930D860ED80DFB0D860E500E630E28
:1000C0004D114D117C117C11BF11F911061406144C
:1000D0001212061407130713DA1306140614F11389
:1000E0000000F0A1F0A229002B00E300E100E000F5
:1000F00000001E00140004001D7435004E001F0097
:100100001A0016001B00007F2A00200008000700CC
:10011000060050002C0021001500090019004F00B6
:100120004B00220017000A0005000000E200230037
:100130002F0000004A0000003E00240030000000B4
:100140004D0000003B0025001C000B0011000000CA
:10015000C200260018000D001000510049002700C1
:100160000C000E003600520028002D0012000F0077
:1001700037000601C1002E00130033003874190146
:100180004C002A0031003400E500E40000000100CA
:10019000010001000100010000003A001E022002DF
:1001A0002202A38001003B001F0221022302010062
:1001B00001003C002F0226022F00010001003D003B
:1001C000300227023000010001003E0031023500FC
:1001D0003502000001003F000100000001000000A6
:1001E000010040000100000001000000010041008A
:1001F00052005100240200000100420024002100AE
:100200001E00010001004300250022001F003700EE
:1002100001004400260023002000270001004500C3
:1002200025022E0231002E004C054600010001007F
:1002300001003D0400000050010001000100010028
:1002400000000100010001000100010001000100A7
:100250000100F2000100010001000100F000F100C6
:100260000100F400010001000100F3000100F500AD
:100270000100010001000100010000000100010077
:100280000100000001000000010001000100000069
:100290000100000001000100010001000100000058
:1002A00001000100010001000100A900010001009E
:1002B00001000100AC00AA00B6000100010001002D
:1002C000AB00A800010001000100010001000100D5
:1002D000010001000100AE00010001000000160352
:1002E0004500720067006F0044006F007800200036
:1002F00045005A00000016034500720067006F00B9
:1003000044006F007800200045005A0000000403FC
:10031000090409026D00040100A0FA0904000001AB
:1003200003010100092111010001223F000705819D
:100330000308000A09040100010301020009211158
:10034000010001224D000705820308000A0904028A
:1003500000010300000009211101000122360007FD
:1003600005830308000A09040300010300000009D3
:100370002111010001223900070584031000011238
:1003800001100100000008EDFE071301000102004A
:100390000105010906A101050719E029E715002556
:1003A0000195087501810205081901290595057552
:1003B000019102950175039101050719002977152F
:1003C000002501957875018102C005010980A10110
:1003D000850216010026B7001A01002AB700751021
:1003E00095018100C0050C0901A1018503160100DA
:1003F000269C021A01002A9C02751095018100C0FA
:1004000005010902A1010901A10005091901290538
:10041000150025019505750181029501750381017E
:100420000501093009311581257F9502750881067E
:1004300009381581257F950175088106050C0A3854
:10044000021581257F950175088106C0C005010947
:1004500006A101050719E029E71500250195087592
:100460000181029501750881010508190129059589
:100470000575019102950175039101050719002980
:10048000FF150025FF950675088100C000000000DB
:1004900000000000000000010204060A0F17202CD3
:1004A0003A4A5D71879DB3C7DAE9F5FCFFFCF5E9CF
:1004B000DAC7B39D87715D4A3A2C20170F0A0604EC
:1004C00002010000000000000000000011241FBE17
:1004D000CFEFDAE0DEBFCDBF04B603FE27C08091C8
:1004E000ED019091EE01A091EF01B091F001873004
:1004F000904BA740B04BD1F41092ED011092EE0159
:100500001092EF011092F00114BE84B7877F84BF70
:100510000FB6F894A8958091600088618093600080
:10052000109260000FBEE0E0FFE3099511E0A0E04B
:10053000B1E0E2E9F6E402C005900D92A433B10700
:10054000D9F721E0A4E3B1E001C01D92AD3EB207AE
:10055000E1F70E9479090C9447230C940000611183
:100560000BC0FC018281882321F085EE0E94E70FF9
:1005700003C085EE0E94AF1080E090E008950895DA
:100580006091B1017091B2018091B3019091B40179
:100590000E94371A56985E9825982D9826982E987E
:1005A00027982F98813019F0823021F00895259AEC
:1005B0002D9A0895269A2E9A089580EC92E0892B20
:1005C00011F00E94C00280E090E0089556985E9875
:1005D00025982D9826982E9827982F988FEF90E0A1
:1005E000909389008093880090938B0080938A0079
:1005F00090938D0080938C00259A2D9A2FEF80E7A1
:1006000092E0215080409040E1F700C00000269A1F
:100610002E9A2FEF80E792E0215080409040E1F742
:1006200000C00000279A2F9A2FEF80E792E0215018
:1006300080409040E1F700C0000025982D982FEFF2
:1006400080E792E0215080409040E1F700C0000038
:1006500026982E982FEF80E792E02150804090401E
:10066000E1F700C0000027982F9856985E982598CB
:100670002D9826982E9827982F98089589EA809388
:10068000800089E08093810024982C983F988AB15B
:100690008F748AB96E98479A8BB1806B8BB9769AB2
:1006A0000E94E6028FEB92E0892B11F00E94BF02BC
:1006B00080E090E0089580E2809300018091340111
:1006C00081110EC00E94AA0381E0809334012FEFB4
:1006D00083ED90E3215080409040E1F700C000009E
:1006E00080E40E94B0038093000181112EC00E941B
:1006F000DA0380930001811128C00E94DA038093FD
:100700000001811122C08FE30E94DA03809300016F
:1007100081111BC00E94D20380E40E94B003809329
:100720000001811112C08CE00E94DA038093000165
:1007300081110BC00E94DA0380930001811105C072
:100740008FE30E94DA03809300010E94D20380911C
:10075000000108951092B9008AE08093B8000895CE
:1007600094EA9093BC009091BC0097FFFCCF9091CD
:10077000B900987F983021F0903111F081E0089510
:100780008093BB0084E88093BC008091BC0087FF0D
:10079000FCCF8091B900887F883111F0803471F7E7
:1007A00080E0089584E98093BC008091BC0084FDC2
:1007B000FCCF08958093BB0084E88093BC008091B7
:1007C000BC0087FFFCCF9091B900987F81E0983200
:1007D00009F480E0089584E88093BC008091BC0017
:1007E00087FFFCCF8091BB000895809100018111AB
:1007F00015C080E40E94B0038093000181110CC0F9
:1008000082E10E94DA0380930001811105C08FEF1D
:100810000E94DA03809300010E94D20384B1807F9A
:1008200084B985B1807F85B98AB1837F8AB98BB15C
:10083000837F8BB93E98469808950E945B0380930E
:1008400000010E94F50380B38C7080BB81B3836F7D
:1008500081BBE4E4F1E0A6E3B1E011921D9281E0F6
:10086000E235F807D1F78EE393E0892B11F00C9471
:100870003E0308959F92AF92BF92CF92DF92EF9284
:10088000FF920F931F93CF93DF93809100018823F2
:1008900079F0809135018F5F80933501811108C017
:1008A0000E945B0380930001811102C00E94E60256
:1008B00086E3E82E81E0F82E8701C0E0D0E0BB247B
:1008C000B39492E0A92ECC24C394D12CC730D10587
:1008D00000F580910001811164C080E40E94B003A2
:1008E00080930001811112C082E10E94DA0380939B
:1008F000000181110BC0C6010C2E01C0880F0A94A3
:10090000EAF780950E94DA03809300010E94D203E7
:1009100048C0CA30A1F028F4C83059F0C93061F09D
:1009200005C0CC3089F070F0CD3089F0209A28983D
:1009300010C0219A29980DC0229A2A980AC0239A99
:100940002B9807C0529A01C0539A5B9802C03E9AF6
:100950004698E0EAEA95F1F78FB181708B25799995
:1009600002C032E001C030E0832B7C9902C034E049
:1009700001C030E0832B7D9902C028E001C020E057
:10098000822B7E9902C090E101C090E0892B9FB13B
:100990009095991F9927991F9295990F907E892B71
:1009A0000FC080910001811150C080E40E94B0030B
:1009B000809300018823B1F1912C0E94D203892DEC
:1009C000D8019C91981719F08C93A09201010E9474
:1009D000F50321960F5F1F4FCE30D10509F076CF7A
:1009E000809101018823B9F081508093010188230F
:1009F00039F0EFE9FFE03197F1F700C000000BC0DC
:100A0000E4E4F1E0D7018D917D018193B4E4EB162C
:100A1000B1E0FB06B9F78DED92E0892BC1F00E94A1
:100A2000DD0215C083E10E94DA0380930001811189
:100A3000C3CF81E40E94B003809300018111BCCF39
:100A40000E94EB03982E9094B8CF80E0B9CF81E05C
:100A5000DF91CF911F910F91FF90EF90DF90CF909A
:100A6000BF90AF909F900895E82FF0E0EC5BFE4FB1
:100A70008081089508958B3B910580F4883A910513
:100A800048F5853A9105D8F48430910508F0B2C054
:100A9000019709F06EC081E090E00895803E9105D5
:100AA00008F467C0883E910508F4A4C09C01205F4B
:100AB00031092031310508F05CC090650895853A10
:100AC000910509F459C0863A910509F058C082E8A9
:100AD00090E40895883A910509F454C0893A910543
:100AE00009F453C08A3A910509F452C08B3A910532
:100AF00009F451C08C3A910509F450C08D3A910522
:100B000009F44FC0803B910509F44EC08E3A91051F
:100B100009F44DC08F3A910509F44CC0813B910511
:100B200009F44BC0823B910509F44AC0833B91050F
:100B300009F449C0843B910509F448C0853B9105FF
:100B400009F447C0863B910509F446C0873B9105EF
:100B500009F445C0883B910509F444C0893B9105DF
:100B600009F443C08A3B910509F442C080E094E453
:100B7000089580E090E0089581E890E4089583E886
:100B800090E4089582EE94E4089589EE94E4089543
:100B90008AEE94E4089585EB94E4089586EB94E45A
:100BA000089587EB94E408958CEC94E408958DEC1B
:100BB00094E4089583E895E408958AE895E4089517
:100BC00082E995E4089584E995E4089581E296E444
:100BD000089583E296E4089584E296E4089585E218
:100BE00096E4089586E296E4089587E296E40895EF
:100BF0008AE296E4089524E5829FC0011124FC0155
:100C000026E0729FE00DF11D1124E60FF11DEE0F9D
:100C1000FF1FEA51FF4F859194910895880F991F06
:100C2000FC01E05AF040859194910895880F991F36
:100C3000FC01E052FF4F85919491089524E5829F35
:100C4000C0011124FC0146E0749FE00DF11D112448
:100C5000E60FF11DEE0FFF1FEA51FF4F85919491B2
:100C60009C013A9521154FE1340708F425C13F5105
:100C70002115304120F49F700E94160608959C01B2
:100C800030532115304118F49927906C089581153F
:100C900020E5920769F40E9428144FEF84E39CE05A
:100CA000415080409040E1F700C000000C942F1BA1
:100CB000813020E5920731F48091CC0181608093EE
:100CC000CC0108959C0130552115304108F05CC0DD
:100CD000292F33272F70332721303105E9F4AC0158
:100CE00064E0440F551F6A95E1F744275370BC0137
:100CF0006370772702C0220F331F6A95E2F73C68C2
:100D0000242B352B73E0880F991F7A95E1F78076B5
:100D10009927822B932B08952230310529F4982F9F
:100D20008827816F906A089523303105A1F4AC01C2
:100D300033E0440F551F3A95E1F7407E57708370BA
:100D4000992721E030E002C0220F331F8A95E2F795
:100D5000C9019C6816C02430310531F5AC0123E08F
:100D6000440F551F2A95E1F7407E577083709927ED
:100D700021E030E002C0220F331F8A95E2F7C9015B
:100D80009A68842B952B08959C013057211530418A
:100D900018F49F70906208959C01305821153041DD
:100DA00018F49F70906A0895803E9105E0F4803CAD
:100DB000910558F58133910509F46FC048F48932E3
:100DC000910509F463C08A32910509F46DC072C0BF
:100DD00089339105E9F082389105D1F08533910589
:100DE00009F44DC067C0833E910581F138F4803E1F
:100DF0009105B9F0823E9105D9F05CC0863E91051F
:100E000061F1873E9105A1F155C00E940E0608953B
:100E10002091DE0120FD02C021FF4CC080EE90E059
:100E200049C08091DE0180FFF9CF89E390E042C0A4
:100E30008091DE0182FF0EC08091DE0184FF03C03D
:100E400080E090E037C083EE90E034C08091DE0116
:100E500082FFF2CF82EE90E02DC08091DE0183FF11
:100E60000BC08091DE0184FDEBCF87EE90E022C0C5
:100E70008091DE0183FFF5CF86EE90E01BC080916C
:100E8000DE0185FF07C089E290E014C08091DE0199
:100E900085FFF9CF85E390E00DC08091DE0186FFEC
:100EA00007C08AE290E006C08091DE0186FFF9CF9C
:100EB00081E390E00E943B0508950895009739F082
:100EC0008A30910514F44D9608950697089587E2A7
:100ED00090E008951F93CF93DF93FC0182818823D4
:100EE00009F440C0C62FD0E0D42B82EE0E94E70F59
:100EF0008D2F82958F7090E00E945E07182F0E94C0
:100F0000E70F812F0E94AF10CE0188279F70892F95
:100F100090E00E945E07182F0E94E70F812F0E9429
:100F2000AF10CE01807F992724E0969587952A956A
:100F3000E1F70E945E07182F0E94E70F812F0E94A1
:100F4000AF10CE018F7099270E945E07C82F0E94B4
:100F5000E70F8C2F0E94AF1082EEDF91CF911F918F
:100F60000C94AF10DF91CF911F9108958091620191
:100F70000895CF93DF9300D01F92CDB7DEB79C01C9
:100F80008091E401843019F593E099833B832A83AF
:100F90009093E9008FEF9091E800815095FD06C095
:100FA00095ED9A95F1F700008111F5CF8091E80059
:100FB00085FF0DC040E050E063E070E0CE01019697
:100FC0000E94260A8091E8008E778093E8000F90B7
:100FD0000F900F90DF91CF910895CF93DF9300D0C2
:100FE0001F92CDB7DEB72091E401243021F522E035
:100FF00029839B838A8383E08093E9008FEF90911C
:10100000E800815095FD06C095ED9A95F1F7000036
:101010008111F5CF8091E80085FF0DC040E050E0E0
:1010200063E070E0CE0101960E94260A8091E800FC
:101030008E778093E8000F900F900F90DF91CF9103
:1010400008959C018091E4018430F9F482E080935A
:10105000E9009FEF8091E800915085FD06C085ED85
:101060008A95F1F700009111F5CF8091E80085FF96
:101070000CC040E050E065E070E0C9010E94260A23
:101080008091E8008E778093E8000895CF93DF93F6
:10109000EC018091E401843009F046C090910C018C
:1010A0009923D9F090910D019923B9F08093E9002B
:1010B0008FEF9091E800815095FD06C095E19A95DB
:1010C000F1F700008111F5CF8091E80085FF2CC079
:1010D00040E050E060E170E017C081E08093E900FB
:1010E0008FEF9091E800815095FD06C095ED9A959F
:1010F000F1F700008111F5CF8091E80085FF14C061
:1011000040E050E068E070E0CE010E94260A809145
:10111000E8008E778093E80080E1FE01A2E5B1E06F
:1011200001900D928A95E1F7DF91CF91089580911A
:10113000E301811109C00E94B70B0E94140C809139
:10114000E20084608093E20008951092E301089524
:1011500008950C9465210E94C51A0E946B210E947B
:10116000BF0E0C945D0742E061EC81E00E94300B01
:1011700042E061EC82E00E94300B42E061EC83E0EF
:101180000E94300B42E161EC84E00C94300B8091C2
:10119000E601833009F455C030F4813071F08230BB
:1011A00009F48EC008958A3009F47AC08B3009F4AE
:1011B00060C0893009F09CC020C08091E501813A6F
:1011C00009F096C08091E800877F8093E8008091C5
:1011D000E9019091EA01892B21F460E182E591E037
:1011E00003C060E080E090E070E00E94710A8091AE
:1011F000E8008B778093E80008958091E5018132C3
:1012000009F076C08091E9019091EA01009719F008
:10121000039709F06DC08091E800877F8093E80014
:101220008091E80082FD05C08091E4018111F8CF32
:101230005FC08091F100809362018091E8008B771C
:1012400053C08091E501813A09F052C08091E901D3
:101250009091EA01892B09F04BC08091E800877FCB
:101260008093E8008091E80080FFFCCF80910C0122
:1012700036C08091E5018132D9F58091E9019091E4
:10128000EA01892BA9F58091E800877F8093E80027
:101290000E94650B8091E70180930C010C94281447
:1012A0008091E501813221F58091E800877F80936C
:1012B000E8000E94650B8091E80180936301089526
:1012C0008091E501813AA1F48091E800877F8093C5
:1012D000E8008091E80080FFFCCF8091630180935B
:1012E000F1008091E8008E778093E8000C94650B04
:1012F000089584B7877F84BF0FB6F894A89580912E
:101300006000886180936000109260000FBE90E0E2
:1013100080E80FB6F89480936100909361000FBE4F
:101320000E940E0F0E94B70B0E94140C8091E200E5
:1013300084608093E20078940E949F0E0E94100FB8
:1013400082E091E00E94BA0E0E9453218091E40154
:10135000853069F40E94871A8091E2018823B1F3F5
:101360000E94B11A882391F30E94100AEFCF0E94C5
:10137000160FECCF292F332723303105C9F060F445
:101380002130310581F02230310509F041C08DE670
:1013900090E022E133E040C021323105E1F0223219
:1013A000310531F135C082E190E02FE733E034C000
:1013B00099278130910549F028F0029749F5EEED23
:1013C000F2E005C0EEE0F3E002C0E6EFF2E0849167
:1013D00090E09F0121C06430D8F4E62FF0E0EE0FDA
:1013E000FF1FEE5DFE4F2081318189E090E014C047
:1013F000643070F470E0FB01EE0FFF1FE65EFE4FFD
:1014000020813181FB01EA5EFE4F808190E004C0C3
:1014100080E090E020E030E0FA01318320830895FD
:1014200080E189BD82E189BD09B400FEFDCF8091D4
:10143000D8008F7D8093D8008091E00082608093F7
:10144000E0008091E00081FDFCCF0895CF92DF9213
:10145000EF92FF920F931F93CF93DF93EC018B01D9
:101460006A010E94840B811133C0C114D10439F088
:10147000F60180819181081B190BC80FD91FE12C3F
:10148000F12C0115110519F18091E80085FD16C0B8
:101490008091E8008E778093E800C114D10449F070
:1014A000F60180819181E80EF91EF182E08285E0EB
:1014B0000FC00E94840B882321F30AC08991809376
:1014C000F10001501109FFEFEF1AFF0ADACF80E0B7
:1014D000DF91CF911F910F91FF90EF90DF90CF9010
:1014E00008952091EB013091EC012617370748F061
:1014F0006115710539F42091E8002E772093E800FA
:1015000001C0B901FC0120E06115710579F18091FC
:10151000E4018823F1F18530F1F18091E80083FD49
:101520003CC08091E80082FD2EC08091E80080FFE1
:10153000EBCF2091F3008091F20090E0922B6115A7
:10154000710551F08830910538F421912093F10014
:10155000615071090196F3CF21E0089709F020E06E
:101560008091E8008E778093E800CECF2111CFCF15
:101570000AC08091E401882361F0853061F0809198
:10158000E80083FD0AC08091E80082FFF2CF80E08E
:10159000089582E0089583E0089581E00895209100
:1015A000EB013091EC012617370748F06115710502
:1015B00039F42091E8002E772093E80001C0B901AA
:1015C000FC0120E06115710591F18091E40188230F
:1015D00009F440C0853009F43FC08091E80083FDE4
:1015E0003DC08091E80082FD2FC08091E80080FF1F
:1015F000E9CF2091F3008091F20090E0922B6115E9
:10160000710559F08830910540F424912093F10040
:101610003196615071090196F2CF21E0089709F0E7
:1016200020E08091E8008E778093E800CBCF2111F5
:10163000CCCF0AC08091E401882361F0853061F04D
:101640008091E80083FD0AC08091E80082FFF2CF1C
:1016500080E0089582E0089583E0089581E0089590
:10166000982F973068F59093E900981739F07091AA
:10167000EC002091ED005091F00003C0242F762F54
:1016800050E021FD02C09F5FECCF3091EB003E7F28
:101690003093EB003091ED003D7F3093ED003091C1
:1016A000EB0031603093EB007093EC002093ED0081
:1016B0005093F0002091EE0027FDE5CF80E00895E3
:1016C0008F708093E90081E008958091E50187FFA4
:1016D00011C08091E80082FD05C08091E401811174
:1016E000F8CF11C08091E8008B770BC08091E401A6
:1016F000882349F08091E80080FFF8CF8091E800CE
:101700008E778093E80008952091E4003091E50001
:1017100095E64091EC00842F817040FF23C08091BA
:10172000E80080FD1DC08091E401882399F0853098
:1017300099F08091EB0085FD11C04091E40050913B
:10174000E5002417350729F3915011F09A01E1CFF4
:1017500084E0089582E0089583E0089581E008958B
:1017600080E008954091E80042FFDDCF08950E9497
:10177000250C0E942D0CE0EEF0E0808181608083DA
:10178000E8EDF0E080818F77808319BCA7EDB0E0B1
:101790008C918E7F8C9380818F7E80831092E30169
:1017A00008950F931F93CF93DF930E94250C0E94FF
:1017B0002D0CC8EDD0E088818F7788838881806880
:1017C000888388818F7D888319BC1092E4011092F0
:1017D000E0011092E2011092E10100EE10E0F80148
:1017E00080818B7F808388818160888342E060E094
:1017F00080E00E94300BE1EEF0E080818E7F8083FC
:10180000E2EEF0E080818160808380818860808367
:10181000F80180818E7F8083888180618883DF9159
:10182000CF911F910F910895E8EDF0E080818F7EB8
:101830008083E7EDF0E080818160808384E082BF77
:1018400081E08093E3010C94D10BE8EDF0E080811E
:101850008E7F80831092E20008951092DA00109239
:10186000E10008951F920F920FB60F9211242F934B
:101870003F934F935F936F937F938F939F93AF9318
:10188000BF93EF93FF938091E10082FF0BC08091A3
:10189000E20082FF07C08091E1008B7F8093E1002E
:1018A0000E949E0E8091DA0080FF1FC08091D800B8
:1018B00080FF1BC08091DA008E7F8093DA008091D8
:1018C000D90080FF0DC080E189BD82E189BD09B4E6
:1018D00000FEFDCF81E08093E4010E94970805C0DF
:1018E00019BC1092E4010E94A5088091E10080FFDC
:1018F00019C08091E20080FF15C08091E2008E7FC8
:101900008093E2008091E20080618093E200809108
:10191000D80080628093D80019BC85E08093E401F0
:101920000E94A9088091E10084FF30C08091E2000C
:1019300084FF2CC080E189BD82E189BD09B400FE2D
:10194000FDCF8091D8008F7D8093D8008091E100F9
:101950008F7E8093E1008091E2008F7E8093E20091
:101960008091E20081608093E2008091E001882311
:1019700011F084E007C08091E30087FD02C081E0A0
:1019800001C083E08093E4010E94AB088091E100F4
:1019900083FF29C08091E20083FF25C08091E10090
:1019A000877F8093E10082E08093E4011092E00160
:1019B0008091E1008E7F8093E1008091E2008E7F34
:1019C0008093E2008091E20080618093E20042E037
:1019D00060E080E00E94300B8091F000886080938E
:1019E000F0000E94A808FF91EF91BF91AF919F91E5
:1019F0008F917F916F915F914F913F912F910F90B8
:101A00000FBE0F901F9018951F920F920FB60F9256
:101A100011242F933F934F935F936F937F938F93F3
:101A20009F93AF93BF93CF93DF93EF93FF93C091B7
:101A3000E900CF708091EC00D82FD17080FDD0E804
:101A40001092E9008091F000877F8093F0007894F5
:101A50000E94480D1092E9008091F0008860809308
:101A6000F000CD2BCF70C093E900FF91EF91DF9193
:101A7000CF91BF91AF919F918F917F916F915F9126
:101A80004F913F912F910F900FBE0F901F9018957F
:101A90001F93CF93DF93CDB7DEB7AA970FB6F89415
:101AA000DEBF0FBECDBFE5EEF1E08091F100819386
:101AB00021E0ED3EF207C9F70E94C7088091E800D7
:101AC00083FF24C18091E5019091E601492F50E008
:101AD0004A30510508F01AC1FA01EA5AFF4F0C9436
:101AE000FC22803881F0823809F010C18091E90130
:101AF0008F708093E9008091EB0085FB882780F947
:101B00001092E90006C08091E1019091E2019111EB
:101B100082609091E800977F9093E8008093F100B5
:101B20001092F100C8C0282F2D7F09F0EFC0882344
:101B300019F0823061F0EAC08091E701813009F04C
:101B4000E5C0933009F080E08093E2012BC08091E2
:101B5000E701811127C08091E9018F7009F4D6C097
:101B60008093E9002091EB0020FF1CC0933021F40A
:101B70008091EB00806214C09091EB009061909393
:101B8000EB0021E030E0A90102C0440F551F8A9507
:101B9000E2F74093EA001092EA008091EB0088603F
:101BA0008093EB001092E9008091E800877F86C067
:101BB0008111ACC01091E7011F778091E30080781C
:101BC000812B8093E3008091E800877F8093E80079
:101BD0000E94650B8091E80080FFFCCF8091E300BC
:101BE00080688093E300111102C082E001C083E0AD
:101BF0008093E4018BC08058823008F087C08091C8
:101C0000E7019091E8018C3D53E0950779F583E079
:101C10008A838AE289834FB7F894DE01139620E025
:101C20003EE051E2E32FF0E050935700E49120FFB3
:101C300003C0E295EF703F5FEF708E2F90E0EA30C7
:101C400010F0C79601C0C0968D939D932F5F2431ED
:101C500049F74FBF8091E800877F8093E8006AE2F0
:101C600070E0CE0101960E94710A14C0AE014F5F70
:101C70005F4F6091E9010E94BA09BC01892B09F408
:101C800045C09091E800977F9093E80089819A8100
:101C90000E94CF0A8091E8008B778093E80036C0DD
:101CA0008038A1F58091E800877F8093E8008091DB
:101CB000E0018093F1008091E8008E778093E80046
:101CC0000E94650B23C0811121C08091E701909192
:101CD000E80199270297D4F48091E800877F8093E8
:101CE000E8008091E7018093E0010E94650B8091FC
:101CF000E001811106C08091E30087FD02C081E010
:101D000001C084E08093E4010E94B3088091E80060
:101D100083FF0AC08091E800877F8093E80080916C
:101D2000EB0080628093EB00AA960FB6F894DEBFBA
:101D30000FBECDBFDF91CF911F9108950895CF932E
:101D40008091E4018823A1F0C091E900CF709091C7
:101D5000EC00892F817090FD80E8C82B1092E9007B
:101D60008091E80083FD0E94480DCF70C093E90088
:101D7000CF91089590936901809368010895E0914F
:101D80006801F0916901309721F00190F081E02D18
:101D9000099480E00895E0916801F091690130971D
:101DA00021F00280F381E02D09940895E09168010B
:101DB000F0916901309721F00480F581E02D0994BC
:101DC000089520916601309167012817390771F055
:101DD0009093670180936601E0916801F091690139
:101DE000309721F00680F781E02D09940895209125
:101DF0006401309165012817390771F090936501EE
:101E000080936401E0916801F0916901309721F0BD
:101E10000084F185E02D0994089508950C940D0F28
:101E20000E94CB1A0E941D040C94911BCF92DF924A
:101E3000EF92FF920F931F93CF93DF93CDB7DEB74F
:101E40002B970FB6F894DEBF0FBECDBF0E943A04A9
:101E50008BE6C82E81E0D82E00E010E0E02E802F27
:101E60000E943405F60141916F01F82EF426B1F479
:101E70000F5F1F4F0E30110589F78FEF89838A831B
:101E80001B820E94D41A8160782F9D838C834981A4
:101E90005A816B818D810E94B90F40C09091CC0115
:101EA00091FF04C08B870E943A058B8520E030E0CB
:101EB0004F2D50E0922FBA01022E02C07595679502
:101EC0000A94E2F760FF24C02E83EF8221E030E025
:101ED000690102C0CC0CDD1C9A95E2F790E08C21E0
:101EE0009D21892B09F420E028870E94D41A816063
:101EF000782F9A8789874E815F8168858A850E94BD
:101F0000B90FF801E559FE4F8081C826C08206C08E
:101F10002F5F3F4F2630310569F6AACF0E94781E09
:101F20000E94BF0E90916A018917A1F00E94BF0E16
:101F300080936A012B960FB6F894DEBF0FBECDBF1B
:101F4000DF91CF911F910F91FF90EF90DF90CF9095
:101F50000C945D072B960FB6F894DEBF0FBECDBF75
:101F6000DF91CF911F910F91FF90EF90DF90CF9075
:101F70000895CF93DF93CDB7DEB72B970FB6F894C4
:101F8000DEBF0FBECDBF4F83588769877A878B87A7
:101F9000DE01119686E0FD0111928A95E9F785E050
:101FA000FE01379601900D928A95E1F749815A8199
:101FB0006B817C818D819E810E94BC162B960FB611
:101FC000F894DEBF0FBECDBFDF91CF910895CF93C0
:101FD000C82F882309F4C1C0823859F40E94BF0E6B
:101FE00081FDBBC089E30E9459190E94111A89E33F
:101FF0000CC0833879F40E94BF0E80FDAEC083E52B
:102000000E9459190E94111A83E50E949819CF91D4
:102010000C94111A843859F40E94BF0E82FD9DC0A1
:1020200087E40E9459190E94111A87E4EECF8CEFC1
:102030008C0F813A48F48C2F0E94B82081118DC0FA
:102040008C2F0E945919E3CF80E28C0F883048F41E
:10205000C77081E001C0880FCA95EAF70E94DA19BB
:10206000D6CF8BE58C0F833078F4C53A29F0C63A89
:1020700031F083E890E005C081E890E002C082E89A
:1020800090E0CF910C94E10E88E58C0F833108F03D
:1020900064C0C83A39F1C93A41F1CA3A49F1CB3A78
:1020A00051F1CC3A59F1CD3A61F1C03B69F1CE3AE8
:1020B00071F1CF3A79F1C13B81F1C23B89F1C33B68
:1020C00091F1C43B99F1C53BA1F1C63BA9F1C73BD6
:1020D000B1F1C83BB9F1C93BC1F1CA3BC9F180E0DC
:1020E00090E038C082EE90E035C089EE90E032C0DA
:1020F0008AEE90E02FC085EB90E02CC086EB90E05C
:1021000029C087EB90E026C08CEC90E023C08DECDA
:1021100090E020C083E891E01DC08AE891E01AC0F9
:1021200082E991E017C084E991E014C081E292E075
:1021300011C083E292E00EC084E292E00BC085E21F
:1021400092E008C086E292E005C087E292E002C019
:102150008AE292E0CF910C94F70ECF9108958823F4
:1021600009F44BC0823859F40E94BF0E81FF45C06C
:1021700089E30E9459190E94111A89E30CC083381F
:1021800071F40E94BF0E80FF38C083E50E94591988
:102190000E94111A83E50E9498190C94111A843830
:1021A00059F40E94BF0E82FF28C087E40E9459198B
:1021B0000E94111A87E4EFCF9CEF980F913A58F3E1
:1021C00090E2980F983050F4877091E001C0990F19
:1021D0008A95EAF7892F0E94E019DFCF9BE5980FD7
:1021E000933020F480E090E00C94E10E885A833123
:1021F00020F480E090E00C94F70E0895882321F0FD
:102200000E94DA190C94111A0895882321F00E9473
:10221000E0190C94111A0895BF92CF92DF92EF92B9
:10222000FF920F931F93CF93DF9300D000D000D085
:10223000CDB7DEB77C0185E0F701DE011196019094
:102240000D928A95E1F7F70183819481892B09F436
:10225000DDC2908181818F3F19F49F3F09F4D6C27E
:10226000F7010281258122952F7099838A838981C4
:102270009A812E830E941819182FB92E0E941719BF
:102280000E94DE17EB2DE295EF704E2F50E0FA0121
:10229000E05AFF4F2E810C94FC228B2D807F9B2DCA
:1022A0009F70F92E882319F0F29480EFF822002312
:1022B00049F0FF2009F457C28F2D0E94EA190E94AD
:1022C000111A51C2812F0E94AF10FF2009F49EC243
:1022D0008F2D0E94F01926960FB6F894DEBF0FBE20
:1022E000CDBFDF91CF911F910F91FF90EF90DF90C5
:1022F000CF90BF900C94111A3B2D307F8B2D8F7097
:10230000303211F08295807F112319F0113021F1C4
:102310002CC00023B9F0222309F490C1213009F028
:102320008DC126960FB6F894DEBF0FBECDBFDF91EC
:10233000CF911F910F91FF90EF90DF90CF90BF90C2
:102340000C94FA19222319F0213009F45FC28E830C
:102350000E94FD198E8186C1002321F0223008F0F1
:1023600055C26CC1211152C27DC1002321F022232C
:1023700009F464C1F8C1222309F474C109C28B2D88
:1023800086958695837019F08130D1F03FC2002385
:1023900021F0812F9B2D937002C080E090E0269663
:1023A0000FB6F894DEBF0FBECDBFDF91CF911F9166
:1023B0000F91FF90EF90DF90CF90BF900C94E10EC3
:1023C000002321F0812F9B2D937002C080E090E0CC
:1023D00026960FB6F894DEBF0FBECDBFDF91CF912A
:1023E0001F910F91FF90EF90DF90CF90BF900C94D2
:1023F000F70E812F002319F00E94801D02C00E9459
:10240000E81D26960FB6F894DEBF0FBECDBFDF9154
:10241000CF911F910F91FF90EF90DF90CF90BF90E1
:102420000C946D1E8B2D837009F075C00111EEC1E7
:10243000812F829586958770880F880F912F9F70C6
:10244000C92ED12CE12CF12C082E04C0CC0CDD1CA3
:10245000EE1CFF1C0A94D2F714FF12C00FE010E02C
:1024600020E030E004C0000F111F221F331F8A95A7
:10247000D2F7C901B801609570958095909503C019
:1024800060E070E0CB014B2D46954695437042309D
:10249000C1F060F56C297D298E299F29413051F1C9
:1024A00026960FB6F894DEBF0FBECDBFDF91CF9159
:1024B0001F910F91FF90EF90DF90CF90BF900C9401
:1024C00005186C297D298E299F2926960FB6F89428
:1024D000DEBF0FBECDBFDF91CF911F910F91FF9057
:1024E000EF90DF90CF90BF900C9421180E940518B8
:1024F000C701B60126960FB6F894DEBF0FBECDBF5A
:10250000DF91CF911F910F91FF90EF90DF90CF90CF
:10251000BF900C94E917002319F08B2D817001C036
:102520008695882309F472C1812F829586958770DC
:10253000880F880F912F9F70C92ED12CE12CF12C80
:10254000082E04C0CC0CDD1CEE1CFF1C0A94D2F734
:1025500014FF12C00FE010E020E030E004C0000FD4
:10256000111F221F331F8A95D2F7C901B801609548
:1025700070958095909503C060E070E0CB014B2D85
:102580004695469543704230C1F060F56C297D292F
:102590008E299F29413051F126960FB6F894DEBF5F
:1025A0000FBECDBFDF91CF911F910F91FF90EF90A4
:1025B000DF90CF90BF900C94DF186C297D298E2975
:1025C0009F2926960FB6F894DEBF0FBECDBFDF91D0
:1025D000CF911F910F91FF90EF90DF90CF90BF9020
:1025E0000C94FB180E94DF18C701B60126960FB69F
:1025F000F894DEBF0FBECDBFDF91CF911F910F9139
:10260000FF90EF90DF90CF90BF900C94C318103FD5
:10261000D1F118F4103E50F4A1C0123F09F463C088
:1026200008F44CC0133F09F473C098C01F708B2D81
:102630008F710023A1F00E945C18812F26960FB69F
:10264000F894DEBF0FBECDBFDF91CF911F910F91E8
:10265000FF90EF90DF90CF90BF900C94FE100E94FF
:102660007D18812F26960FB6F894DEBF0FBECDBF22
:10267000DF91CF911F910F91FF90EF90DF90CF905E
:10268000BF900C9405110023A9F02111BFC08B2D20
:102690008F7126960FB6F894DEBF0FBECDBFDF91C7
:1026A000CF911F910F91FF90EF90DF90CF90BF904F
:1026B0000C94A218223008F0A9C0E9CF0023A9F099
:1026C0008B2D8F7126960FB6F894DEBF0FBECDBF4F
:1026D000DF91CF911F910F91FF90EF90DF90CF90FE
:1026E000BF900C945C18002359F38B2D8F712696A4
:1026F0000FB6F894DEBF0FBECDBFDF91CF911F9113
:102700000F91FF90EF90DF90CF90BF900C947D18C9
:10271000002399F08B2D8F7126960FB6F894DEBFAB
:102720000FBECDBFDF91CF911F910F91FF90EF9022
:10273000DF90CF90BF900C94471826960FB6F89470
:10274000DEBF0FBECDBFDF91CF911F910F91FF90E4
:10275000EF90DF90CF90BF900C943D180023A9F02C
:10276000222309F4ADCF812F26960FB6F894DEBF51
:102770000FBECDBFDF91CF911F910F91FF90EF90D2
:10278000DF90CF90BF900C94E70F222309F4ADCFD8
:10279000812F26960FB6F894DEBF0FBECDBFDF9116
:1027A000CF911F910F91FF90EF90DF90CF90BF904E
:1027B0000C94AF104B2D4F70612FC7010E94AF02D8
:1027C00026960FB6F894DEBF0FBECDBFDF91CF9136
:1027D0001F910F91FF90EF90DF90CF90BF900C94DE
:1027E00061174B2D4F70612FC70126960FB6F894D5
:1027F000DEBF0FBECDBFDF91CF911F910F91FF9034
:10280000EF90DF90CF90BF900C946A0726960FB69A
:10281000F894DEBF0FBECDBFDF91CF911F910F9116
:10282000FF90EF90DF90CF90BF9008950E94F7192E
:102830000E94CC190E94111A0E941D1F0E946D1E39
:1028400080E090E00E94E10E80E090E00C94F70EB2
:102850000E94E7190C9416140E941819292F22952A
:102860002F702C3030F42A3048F42250223078F483
:1028700005C02C3041F02F3031F009C0803E48F0C7
:10288000803F29F406C093FB882780F9089580E0F3
:10289000089581E00895CF93DF9300D000D01F9278
:1028A000CDB7DEB70F900F900F900F900F90DF9184
:1028B000CF910895CF93DF9300D000D000D0CDB753
:1028C000DEB726960FB6F894DEBF0FBECDBFDF9100
:1028D000CF9108951F93CF93DF93C091790116E0B4
:1028E00080917A01C81799F0D0E01C9FF0011D9FDC
:1028F000F00D1124E558FE4F4081518162817381B2
:10290000848195810E945A142196C770E9CFDF9186
:10291000CF911F9108954091AB015091AC0160910E
:10292000AD017091AE018091AF019091B0010C9416
:102930005A148091B00182958F7009F054C0809133
:10294000AD01882309F44FC080917901A0917A01EB
:102950004091AE015091AF016091AB017091AC011B
:10296000B6E08A1709F43FC090E041155105C1F166
:102970007F3F11F46F3FA1F1B89FF001B99FF00DB7
:102980001124E558FE4F218127132AC020812613E8
:1029900027C02281211124C02381348124173507C7
:1029A00010F421503109241B350B283C3105C0F4AB
:1029B0002091B0012F7020612093B00126E0289F64
:1029C000F001299FF00D1124E058FE4F80818F7097
:1029D000806180838BEA91E00E940C110C946A1450
:1029E00001968770BECF0895CF92DF92EF92FF924B
:1029F0000F931F93CF93DF93CDB7DEB762970FB6D8
:102A0000F894DEBF0FBECDBF8C0185E0F801DE017A
:102A10001D9601900D928A95E1F7D8014C9111967F
:102A20005C91119712966C918091AE019091AF01DB
:102A3000009709F475C13091AB017091AC017F3FF3
:102A400019F43F3F09F46CC1F801C380D480E090D1
:102A5000AD01EE2009F4BEC02091B001C816D90620
:102A600028F0D601A81BB90BCD0104C08095909524
:102A70008C0D9D1DFF24F394883C910578F0F12C7A
:102A8000207F09F0C4C07C2DD98AC88A89890E9418
:102A90004B148BEA91E00E940C11AFC0822F807F13
:102AA00009F045C0571313C0431311C061110FC083
:102AB0002F7020612093B0010E948B148BEA91E06B
:102AC0000E940C118091B001F80185832EC0CD28A1
:102AD00019F15F3F11F44F3FF9F0F62E61111CC060
:102AE0008091790120917A0136E0821709F45BC068
:102AF00090E0389FF001399FF00D1124E558FE4F0A
:102B00007181571306C07081471303C07281711120
:102B100003C001968770E9CFF62E662309F41CC125
:102B20008091B00181608093B001F12C15C15713E1
:102B300009C0431307C0611105C08091B001F801BD
:102B40008583C8C04D875E878D859E856A8B0E9470
:102B50002C146A898823D1F16623C1F12091B00138
:102B6000822F82958F7090E0029774F08091AB0174
:102B70009091AC0198878F831986DB86CA862C8753
:102B8000CE0107960E940C1186E0F801ABEAB1E095
:102B900001900D928A95E1F70E9499140E948B147E
:102BA000FF24F394D9C04D875E878D859E850E9452
:102BB0001819292F22952F70223008F0C1C09F705C
:102BC00009F0BBC0805E883008F4C6C0C8010E940E
:102BD0000C11E6CFC816D90608F453C0F601E81B5D
:102BE000F90BCF01883C910508F450C0F12C7C2DE5
:102BF000D98AC88A89890E944B14EBEAF1E086E001
:102C0000DF011D928A95E9F70E948B14A5C0571326
:102C100014C0431312C0611110C08091B001F801BB
:102C20008583C8010E940C1186E0EBEAF1E0DF0128
:102C30001D928A95E9F7FE2C8FC04D875E878D85A2
:102C40009E856A8B0E942C146A89882309F4BECF62
:102C5000662309F4BBCF2091B001822F82958F703B
:102C600090E002970CF490CF8091AB019091AC0171
:102C70009A8389831B82DD82CC822E83CE010196CA
:102C800081CF809590958C0D9D1DACCFF62E66233F
:102C900009F49CCF571333C0431331C02091B001C6
:102CA00020FD24C0822F82958F70482F50E041155F
:102CB0005105E1F0D80115962C9315974F30510529
:102CC00049F08F5F982F9295907F822F8F70892B7C
:102CD00015968C93C8010E940C1186E0F801ABEAAE
:102CE000B1E001900D928A95E1F78ECF86E0F80170
:102CF000ABEAB1E001900D928A95E1F72DC04D87C6
:102D00005E878D859E850E942C1481113DCF809118
:102D1000B00181608093B001C8010E940C111CC0F9
:102D2000662309F453CF4D875E878D859E850E946B
:102D30002C14882309F44ACF27CF811143CF0CC02C
:102D4000243008F043CF9F7009F43CCFD80115968A
:102D50009C91907F09F036CF8F2D62960FB6F89434
:102D6000DEBF0FBECDBFDF91CF911F910F91FF90BE
:102D7000EF90DF90CF9008951F93CF93DF93CDB75F
:102D8000DEB72C970FB6F894DEBF0FBECDBF4F83D2
:102D9000588769877A878B879C87CE0107960E9420
:102DA000F414882371F08A859B85892B09F441C02E
:102DB00088858F3F09F065C08F818F3F09F061C022
:102DC00038C086E0FE013796DE01119601900D9223
:102DD0008A95E1F76A857B856115710551F1FF815F
:102DE000E885EF3F11F4FF3F21F120917A0130E0B7
:102DF000C9010196877099274091790150E08417A5
:102E0000950709F447C0F983EA837D836C8396E0D4
:102E1000929FD001939FB00D1124A558BE4FFE0183
:102E2000319601900D929A95E1F780937A010E9474
:102E30006A1416E08091790190917A018917B9F1AD
:102E4000189FC001112485589E4F0E94F4148823B6
:102E500071F1E09179011E9FF0011124E558FE4FB8
:102E60004081518162817381848195810E945A14CD
:102E70008091790190E0019687709927809379017C
:102E8000D9CF4F81588569857A858B859C850E942D
:102E90005A14CFCF0E94281410927A01109279010F
:102EA000EBEAF1E086E0DF011D928A95E9F72C96C6
:102EB0000FB6F894DEBF0FBECDBFDF91CF911F914B
:102EC0000895EF92FF920F931F93CF93DF938C019E
:102ED000892B09F46CC0F12CEE24E394E8012196CF
:102EE000F8018491843740F4843008F051C0813077
:102EF00081F0823019F15BC0853709F444C0A8F134
:102F00009CE7980F903708F052C08F770E94AF105F
:102F100041C00E5F1F4FFE01849190E2980F9830E0
:102F200050F48770FE2D01C0FF0F8A95EAF78F2FAE
:102F30000E94EA1914C00E94E70F2DC00E5F1F4FB8
:102F4000FE01849190E2980F983060F48770FE2D16
:102F500001C0FF0F8A95EAF78F2F0E94F0190E9497
:102F6000111A19C00E94AF1016C00E5F1F4FFE014C
:102F7000C491CC2381F08FE99FE00197F1F700C065
:102F80000000C150F6CF0E5F1F4FFE01F49003C04A
:102F90000E94E70F8E018F2D882309F49FCFEFE960
:102FA000FFE03197F1F700C000008150F5CFDF91CD
:102FB000CF911F910F91FF90EF9008950895609326
:102FC000B5017093B6018093B7019093B8010C944A
:102FD00016140F931F930091B5011091B601209123
:102FE000B7013091B801DC01CB01802B912BA22BD2
:102FF000B32B8093B5019093B601A093B701B09322
:10300000B8011F910F910C9416140F931F93009108
:10301000B5011091B6012091B7013091B801DC01E2
:10302000CB0180239123A223B3238093B5019093F6
:10303000B601A093B701B093B8011F910F910C9402
:1030400016140F931F930091B5011091B6012091B2
:10305000B7013091B801DC01CB0180279127A2276D
:10306000B3278093B5019093B601A093B701B093B5
:10307000B8011F910F910C9416141092B101109287
:10308000B2011092B3011092B4010C94161441E0F5
:1030900050E060E070E004C0440F551F661F771FCA
:1030A0008A95D2F74093B1015093B2016093B30176
:1030B0007093B4010C94161441E050E060E070E0AD
:1030C00004C0440F551F661F771F8A95D2F7809161
:1030D000B1019091B201A091B301B091B401482B1C
:1030E000592B6A2B7B2B4093B1015093B201609313
:1030F000B3017093B4010C94161441E050E060E009
:1031000070E004C0440F551F661F771F8A95D2F7E1
:1031100040955095609570958091B1019091B20164
:10312000A091B301B091B401482359236A237B23B2
:103130004093B1015093B2016093B3017093B40115
:103140000C94161441E050E060E070E004C0440FBD
:10315000551F661F771F8A95D2F78091B101909114
:10316000B201A091B301B091B401482759276A2751
:103170007B274093B1015093B2016093B3017093E8
:10318000B4010C9416140F931F930091B101109188
:10319000B2012091B3013091B401DC01CB01802B4D
:1031A000912BA22BB32B8093B1019093B201A093EA
:1031B000B301B093B4011F910F910C9416140F93A7
:1031C0001F930091B1011091B2012091B301309190
:1031D000B401DC01CB0180239123A223B32380938C
:1031E000B1019093B201A093B301B093B4011F91C8
:1031F0000F910C9416140F931F930091B10110912D
:10320000B2012091B3013091B401DC01CB018027E0
:103210009127A227B3278093B1019093B201A09385
:10322000B301B093B4011F910F910C94161408953B
:10323000CF92DF92EF92FF920F931F93CF93DF9382
:103240008C01C090B101D090B201E090B301F09038
:10325000B4018091B5019091B601A091B701B091F0
:10326000B801C82AD92AEA2AFB2ACFE1D0E0D7013F
:10327000C6010C2E04C0B695A795979587950A941C
:10328000D2F780FF07C0B8018C2F0E941E06813044
:10329000910531F4219758F7B80180E00E941E068D
:1032A000DF91CF911F910F91FF90EF90DF90CF9022
:1032B000089590910C019923F1F090910D019923BB
:1032C000D1F0982F9695969596959F3080F5E09140
:1032D0000E01F0910F01E90FF11D877021E030E040
:1032E000A90102C0440F551F8A95E2F7CA019181D6
:1032F000892B8183089520910E0130910F01F901EE
:1033000032969FEF40E05191851789F09F3F19F465
:10331000511101C0942F4F5F4E30A9F79F3F39F0F4
:10332000F901E90FF11D97FDFA958283089508953B
:1033300090910C019923F9F090910D019923D9F006
:10334000982F9695969596959F3028F5E0910E01C9
:10335000F0910F01E90FF11D877021E030E0A90124
:1033600002C0440F551F8A95E2F7CA0180959181EA
:1033700089238183089520910E0130910F01F90175
:103380003296205F3F4F9081891301C010823196A1
:10339000E217F307C1F7089581E090E0E0910E0194
:1033A000F0910F01E80FF91F10820196803191050D
:1033B000A9F708959091CB01892B8093CB010895B3
:1033C00080959091CB0189238093CB010895109231
:1033D000CB0108959091CA01892B8093CA01089569
:1033E00080959091CA0189238093CA010895109213
:1033F000CA0108958093B90108951092B901089502
:1034000080910E0190910F01FC0131969C01205F8B
:103410003F4F80E0919191118F5FE217F307D1F751
:103420000895E0910E01F0910F018091CB0180830E
:10343000E0910E01F0910F0190818091CA01892BDA
:1034400080838091B901882361F0E0910E01F091B1
:103450000F019081892B80830E94001A81111092A4
:10346000B90180910E0190910F010C94CB0ECF9277
:10347000DF92EF92FF926C01EE24FF24C114D1047D
:10348000E104F10421F0C701B60120E101C020E010
:10349000C72ED82EE92EFF24C114D104E104F10473
:1034A00019F0285FC701B6016B017C0154E0F69466
:1034B000E794D794C7945A95D1F7C114D104E10485
:1034C000F10419F02C5FC701B6016B017C0142E0E9
:1034D000F694E794D794C7944A95D1F7C114D104D0
:1034E000E104F10419F02E5FC701B601DC01CB0144
:1034F000B695A79597958795892B8A2B8B2B09F0E5
:103500002F5F822FFF90EF90DF90CF9008958091F2
:10351000E401843011F120E488E190E00FB6F894E2
:10352000A895809360000FBE2093600083B7817FD1
:10353000846083BF83B7816083BF7894889583B7A5
:103540008E7F83BF0FB6F894A89580916000886144
:1035500080936000109260000FBE089508950C944F
:10356000AE1ACF930E94AF1A0E943A040E94AE1A7C
:10357000C0E08C2F0E943405811104C0CF5FCE3093
:10358000C1F701C081E0CF9108950E9428140E94E4
:10359000BF0E0C945D0782E084BD93E095BD9AEF69
:1035A00097BD80936E0008952FB7F8948091CD0158
:1035B0009091CE01A091CF01B091D0012FBF08957D
:1035C000CF92DF92EF92FF920F931F932FB7F89451
:1035D0004091CD015091CE016091CF017091D00109
:1035E0002FBF6A017B01EE24FF248C0120E030E034
:1035F000C016D106E206F30610F4415051099A01B3
:10360000281B390BC9011F910F91FF90EF90DF909C
:10361000CF9008951F920F920FB60F9211248F939F
:103620009F93AF93BF938091CD019091CE01A091D4
:10363000CF01B091D0010196A11DB11D8093CD01A4
:103640009093CE01A093CF01B093D001BF91AF91E1
:103650009F918F910F900FBE0F901F9018950E9411
:10366000B70BF8942FEF87EA91E621508040904005
:10367000E1F700C0000087E090EBDC018093ED01F2
:103680009093EE01A093EF01B093F0019CE088E1EC
:103690000FB6F894A895809360000FBE90936000D9
:1036A000FFCFEF92FF920F931F93CF93DF93D82F0B
:1036B000C0E08C2F0E94340500E010E0E82EF12CD1
:1036C000C701002E02C0959587950A94E2F780FD08
:1036D00006C00F5F1F4F0630110591F709C0602F1C
:1036E0007C2F80E00E94FB058D13F3CF81E004C0A6
:1036F000CF5FCE30F1F680E0DF91CF911F910F9137
:10370000FF90EF900895CF93C82F8CE20E94511B39
:10371000882321F08C2FCF910C94511B80E0CF9106
:103720000895CF930E94D81C811102C00E94BE1C34
:10373000C5E6C15049F00E943A048FE39CE9019725
:10374000F1F700C00000F5CF89E20E94831B8111D0
:1037500013C18AE20E94831B81110E94BE1C85E076
:103760000E94831B81110E942F1B0E94E31C8093E7
:10377000CC0187E00E94831B8823A9F18BE10E9482
:10378000831B882351F08091CC0181FB222720F9F3
:1037900091E0922790FB81F90EC08EE00E94831B7E
:1037A000882361F08091CC0182FB222720F991E0EF
:1037B000922790FB82F98093CC0115C080E10E9492
:1037C000831B9091CC01882341F093FB222720F9A1
:1037D00081E0822780FB93F904C0892F809580FBCC
:1037E00090F99093CC018091CC010E94E71C0E943B
:1037F000F51C8093DE0180EE0E94831B882341F03C
:103800008091DE01982F909590FB80F98093DE01E6
:1038100089E30E94831B882359F08091DE0181FB9C
:10382000222720F991E0922790FB81F98093DE0115
:1038300082EE0E94831B882359F08091DE0182FB77
:10384000222720F991E0922790FB82F98093DE01F4
:1038500086EE0E94831B882359F08091DE0183FB52
:10386000222720F991E0922790FB83F98093DE01D3
:1038700083EE0E94831B882359F08091DE0184FB34
:10388000222720F991E0922790FB84F98093DE01B2
:1038900085E30E94831B882359F08091DE0185FB1C
:1038A000222720F991E0922790FB85F98093DE0191
:1038B00081E30E94831B882359F08091DE0186FBFF
:1038C000222720F991E0922790FB86F98093DE0170
:1038D00081E10E94831B882359F08091DE0187FBE0
:1038E000222720F991E0922790FB87F98093DE014F
:1038F0008091DE010E94F91C8091DE0187FB882700
:1039000080F980930D0187E20E94831BC82F8EE10E
:103910000E94831B8111C2608FE10E94831B811171
:10392000C46080E20E94831B8111C86081E20E9412
:10393000831B8111C06182E20E94831B8111C062DE
:1039400083E20E94831B8111C06484E20E94831B76
:10395000882311F0C06802C0CC2329F08C2F0E946C
:10396000F01C6C2F03C00E94EC1C682F70E080E0FC
:1039700090E0CF910C94DF17CF9108956DEE7EEF1C
:1039800080E090E00E94322360E082E090E00E94BC
:10399000242360E083E090E00E94242360E084E040
:1039A00090E00E94242360E085E090E00C942423C2
:1039B00080E090E00E941E2321E08D3E9E4F09F0A2
:1039C00020E0822F089582E090E00C941623682F67
:1039D00082E090E00C94242383E090E00C94162382
:1039E000682F83E090E00C94242384E090E00C9412
:1039F0001623682F84E090E00C9424238091D30157
:103A000080FF0BC06091130185E0689FB001112415
:103A100075956795759567952BC081FF09C0609175
:103A2000130185E0689FB00111247595679520C04A
:103A300082FF07C06091130185E0689FB0011124E7
:103A400017C09091D4019923D1F06091120196177B
:103A500088F72091130185E0289F90011124929FFF
:103A6000A001939F500D112470E0CA010E94E8222A
:103A70006038710540F46115710519F406C065E000
:103A800070E0862F08958FE7089581E00895809172
:103A9000D30180FF08C06091110170E075956795B2
:103AA0007595679521C081FF06C06091110170E096
:103AB0007595679519C082FF04C06091110170E08F
:103AC00010C09091D401992399F06091100196173C
:103AD000A0F780911101899FC001112470E00E941C
:103AE000E8226038710540F46115710519F406C0CB
:103AF00061E070E0862F08958FE7089581E00895D2
:103B0000803F21F40E94FE1C819504C0813F29F46E
:103B10000E94FE1C8093D7010895823F21F40E94E9
:103B2000FE1C819504C0833F29F40E94FE1C8093F3
:103B3000D6010895893F19F40E94471D05C08A3FA8
:103B400031F40E94471D81958093D80108958B3FE1
:103B500021F40E94471D819504C08C3F29F40E94E6
:103B6000471D8093D9010895843F21F48091D501A8
:103B7000816017C0853F21F48091D501826011C01A
:103B8000863F21F48091D50184600BC0873F21F4EA
:103B90008091D501886005C0883F31F48091D501BE
:103BA00080618093D50108958D3F21F48091D301E8
:103BB00081600BC08E3F21F48091D301826005C0EB
:103BC0008F3F29F48091D30184608093D3010895BD
:103BD000803F39F48091D70187FF6CC01092D701E4
:103BE00069C0813F29F48091D7011816BCF362C0E7
:103BF0009091D601823F29F497FF5CC01092D601C4
:103C000059C0833F19F41916CCF354C0893F41F4CD
:103C10008091D80118160CF04DC01092D8014AC0FE
:103C20008A3F29F48091D80187FF44C0F6CF8B3FAB
:103C300039F48091D90187FF3DC01092D9013AC073
:103C40008C3F29F48091D9011816BCF333C0843F0E
:103C500021F48091D5018E7F17C0853F21F480919A
:103C6000D5018D7F11C0863F21F48091D5018B7FD6
:103C70000BC0873F21F48091D501877F05C0883F25
:103C800031F48091D5018F7E8093D50113C08D3F93
:103C900021F48091D3018E7F0BC08E3F21F480915F
:103CA000D3018D7F05C08F3F29F48091D3018B7F95
:103CB0008093D3018091D60181110EC08091D701EC
:103CC00081110AC08091D801811106C08091D9016B
:103CD000811102C01092D401089585ED91E00E94F7
:103CE000D60E0E94D41A9093D2018093D1010895E8
:103CF0001F93CF93DF938091D1019091D2010E94C5
:103D0000E01AAC019091D401992321F02091140183
:103D100030E006C0209115018AE0289F900111240F
:103D20004217530708F485C08091D601C091D7018E
:103D3000D091D8011091D901811107C0C11175C06E
:103D4000D11173C0111171C074C09F3F19F09F5FF2
:103D50009093D401181624F40E94FE1C8093D6017F
:103D60008091D60187FF05C00E94FE1C819580933B
:103D7000D6011C1624F40E94FE1C8093D70180916A
:103D8000D70187FF05C00E94FE1C81958093D70153
:103D90006091D601662331F1C091D701CC2311F196
:103DA000062E000C770B880B990B0E94EF2123E362
:103DB00033E343E35FE30E9453220E94B721609301
:103DC000D6016C2FCC0F770B880B990B0E94EF213B
:103DD00023E333E343E35FE30E9453220E94B721CE
:103DE0006093D7011D1624F40E94471D8093D801CB
:103DF0008091D80187FF05C00E94471D819580935F
:103E0000D801111624F40E94471D8093D901809196
:103E1000D90187FF05C00E94471D81958093D90174
:103E2000DF91CF911F910C946D1E9F3F09F08FCFB2
:103E3000A0CFDF91CF911F910895E5EDF1E085E0EE
:103E4000DF011D928A95E9F71092D4011092D301F7
:103E50000895833081F128F4813059F08230D1F017
:103E60000895853009F449C0B8F1863009F456C088
:103E7000089580911501262F30E0280F311D2F3F26
:103E8000310524F4680F6093150108958FEF809336
:103E90001501089580911401262F30E0280F311D5F
:103EA0002F3F310524F4680F6093140108958FEFBC
:103EB00080931401089580911301262F30E0280F7C
:103EC000311D2F3F310524F4680F609313010895CD
:103ED0008FEF80931301089580911201262F30E017
:103EE000280F311D2F3F310524F4680F6093120114
:103EF00008958FEF80931201089580911101262F6C
:103F000030E0280F311D2F3F310524F4680F6093F6
:103F1000110108958FEF8093110108958091100190
:103F2000262F30E0280F311D2F3F310524F4680F74
:103F30006093100108958FEF8093100108958330EE
:103F400011F128F4813049F0823091F008958530E4
:103F500081F120F18630C1F1089580911501681733
:103F600020F4861B80931501089510921501089581
:103F700080911401681720F4861B80931401089522
:103F800010921401089580911301681720F4861B84
:103F900080931301089510921301089580911201E6
:103FA000681720F4861B8093120108951092120165
:103FB000089580911101681720F4861B80931101E8
:103FC000089510921101089580911001681720F44E
:103FD000861B8093100108951092100108950F938D
:103FE0001F938D3109F46BC008F03FC08E3009F487
:103FF0007DC0C0F4873009F46EC068F4863009F0E3
:10400000AFC08091CC01817F8E7F8093CC0181E015
:104010008093DB01A6C0883009F458C08B3009F4C6
:104020009BC09EC0863109F497C078F4803109F4B2
:1040300070C0813109F094C00E94281490910D0144
:1040400081E0892780930D0187C0893109F484C0FC
:104050008B3109F085C08091CC0181FB222720F9AA
:1040600091E0922790FB81F94AC0853309F45BC047
:1040700048F4873209F457C008F45AC0893209F469
:1040800052C06EC0833438F48A3308F067C0883376
:1040900009F462C065C0833409F445C0883409F06E
:1040A0005FC00E9428140FEF13ED20E30150104071
:1040B0002040E1F700C000000E942F1B4DC00E946D
:1040C00071210E94BF0E0E945D0746C00E94E31C42
:1040D0000E94F51C41C09091CC01892F817090FF06
:1040E00012C0917F9E7F9093CC013BC08091CC0108
:1040F00082FB222720F991E0922790FB82F980939E
:10410000CC01992349F18091CC0181608093CC014D
:1041100023C08091CC0183FB222720F991E09227D4
:1041200090FB83F9ECCF61E070E080E090E010C09C
:104130008D5141E050E060E070E08A019B0104C0D5
:10414000000F111F221F331F8A95D2F7C901B80132
:104150000E94DF170E94281481E003C08953E9CF31
:1041600080E01F910F91089580E008950C94B42091
:10417000CF93C82F8091DB01813079F018F0823025
:10418000E9F187C0E0910E01F0910F01808181314A
:1041900069F0823209F07FC009C0E0910E01F09110
:1041A0000F018081813111F0823261F48C2F0E94E5
:1041B000B620811104C08C2F0E94EF1F1DC081E02A
:1041C00090E01AC08C2F0E94B420811114C0C43119
:1041D00079F048F4CB3079F0C03109F060C082E06A
:1041E0008093DB0108C0C93219F0C83321F057C0F1
:1041F0001092DB0154C081E0817053C0C93289F153
:1042000018F5C43171F1A8F4C73009F046C08AE04E
:104210008093150194E19093140193E0909313011E
:104220008093120188E08093110188E2809310014D
:1042300034C0CE51C63088F5EC2FF0E0E65DFE4F7D
:1042400080818093DA0129C0CE34E9F020F4CB34A8
:1042500021F56AE013C0C13579F0C235F1F461E0AF
:104260000DC08091DA01882319F01092DA0115C08F
:1042700081E08093DB0115C061E006C08091DA0126
:104280000E94291F0AC06AE08091DA010E949F1FE4
:1042900004C01092DB0180E004C081E002C080E035
:1042A000ABCFCF910895E1E8F0E080818860808312
:1042B0008081816080838FB7F89493E09093890028
:1042C00090ED909388008FBF0895EFE6F0E0808135
:1042D000826080830895EFE6F0E080818D7F8083A7
:1042E0000895EFE6F0E0908182E0892780830895C9
:1042F0001F920F920FB60F9211242F933F934F935B
:104300005F936F937F938F939F93AF93BF93EF933D
:10431000FF938091DC019091DD0101969093DD0186
:104320008093DC01811103C082E00E945D07E0916F
:10433000DD01E695E695F0E0E457FB4FE4918091CE
:10434000DC018E1303C080E00E945D07FF91EF91B6
:10435000BF91AF919F918F917F916F915F914F919D
:104360003F912F910F900FBE0F901F9018950E94B4
:10437000BE216894B1110C944D2208950E943222FE
:1043800088F09F5798F0B92F9927B751B0F0E1F016
:10439000660F771F881F991F1AF0BA95C9F714C0C6
:1043A000B13091F00E944C22B1E008950C944C225F
:1043B000672F782F8827B85F39F0B93FCCF38695FF
:1043C00077956795B395D9F73EF49095809570955C
:1043D00061957F4F8F4F9F4F0895E89409C097FBD9
:1043E0003EF490958095709561957F4F8F4F9F4FCC
:1043F0009923A9F0F92F96E9BB279395F695879510
:1044000077956795B795F111F8CFFAF4BB0F11F4D2
:1044100060FF1BC06F5F7F4F8F4F9F4F16C0882379
:1044200011F096E911C0772321F09EE8872F762FAF
:1044300005C0662371F096E8862F70E060E02AF0F0
:104440009A95660F771F881FDAF7880F96958795DC
:1044500097F9089557FD9058440F551F59F05F3F45
:1044600071F04795880F97FB991F61F09F3F79F096
:1044700087950895121613061406551FF2CF469518
:10448000F1DF08C0161617061806991FF1CF86959A
:104490007105610508940895E894BB27662777277E
:1044A000CB0197F908950E9466220C94D7220E94AE
:1044B000C92238F00E94D02220F0952311F00C94EC
:1044C000C0220C94C62211240C944D220E942A2250
:1044D00070F3959FC1F3950F50E0551F629FF00157
:1044E000729FBB27F00DB11D639FAA27F00DB11D70
:1044F000AA1F649F6627B00DA11D661F829F2227F9
:10450000B00DA11D621F739FB00DA11D621F839F7F
:10451000A00D611D221F749F3327A00D611D231F55
:10452000849F600D211D822F762F6A2F11249F57A3
:1045300050409AF0F1F088234AF0EE0FFF1FBB1FA6
:10454000661F771F881F91505040A9F79E3F510565
:1045500080F00C94C0220C944D225F3FE4F3983E0F
:10456000D4F3869577956795B795F795E7959F5F0F
:10457000C1F7FE2B880F911D9695879597F90895A1
:1045800097F99F6780E870E060E008959FEF80EC06
:10459000089500240A9416161706180609060895A9
:1045A00000240A9412161306140605060895092E0F
:1045B0000394000C11F4882352F0BB0F40F4BF2B7E
:1045C00011F460FF04C06F5F7F4F8F4F9F4F0895BE
:1045D00097FB072E16F4009407D077FD09D00E94B0
:1045E000022307FC05D03EF4909581959F4F0895D6
:1045F000709561957F4F0895EE0FFF1F0590F49120
:10460000E02D0994AA1BBB1B51E107C0AA1FBB1FC9
:10461000A617B70710F0A61BB70B881F991F5A954E
:10462000A9F780959095BC01CD010895F999FECF29
:1046300092BD81BDF89A992780B50895A8E1B0E0B0
:1046400042E050E00C943923262FF999FECF1FBA8F
:1046500092BD81BD20BD0FB6F894FA9AF99A0FBEAB
:10466000019608950E942423272F0C942523DC0112
:10467000CB01FC01F999FECF06C0F2BDE1BDF89A6D
:10468000319600B40D9241505040B8F70895F89417
:02469000FFCF5A
:104692002002B60746082108ED07B9070101BA0151
:1046A20028080A03140A3F4D36394D040004CA0390
:1046B200910324033D0356036F030102030405061D
:0446C20007080900DC
:00000001FF
